:100000004CC066C065C064C063C062C061C060C0EF
:100010005FC0F8C65DC05CC05BC05AC059C058C064
:1000200057C056C055C087C186C185C184C183C130
:10003000DDC281C1DBC282C2D9C2F1C1F0C1D6C268
:10004000EEC1EDC1D3C2D2C2D1C2A0C2AFC20000C4
:1000500037343100003835320000363330040404C0
:100060000404040404020202020202030303030361
:10007000030102040810204080010204081020013E
:10008000020408102000000000000000000003042B
:100090000500000000000000000011241FBECFE595
:1000A000D4E0DEBFCDBF10E0A0E6B0E0EAE1F1E1D0
:1000B00002C005900D92A036B107D9F710E0A0E676
:1000C000B0E001C01D92AE39B107E1F797D624C860
:1000D00097CF84E190E090939900809398000895E1
:1000E0000F931F93880F991F672B49F08C010659B6
:1000F0001F4F60E0F80180816BD761E008C08C0180
:1001000006591F4F61E0F801808162D760E0F80175
:1001100080810AD71F910F9108950F931F93CF935A
:10012000DF93EC018B018091680090916900892B2D
:1001300009F4DEC0C830D1055CF4C430D10594F4B4
:10014000209709F45BC0C130D10509F04FC284C0CB
:10015000CE30D10539F0C331D10541F02B9709F0EC
:1001600045C21FC0B801CE01BBDF40C280919400E0
:1001700090919500892B09F039C260E083E028D77F
:1001800061E070E080E090E079D62FE141E062E04C
:1001900081E053D761E070E080E090E06FD6202FDF
:1001A0001BC0672B31F181E090E090939500809324
:1001B000940060E083E00CD761E070E080E090E0C4
:1001C0005DD62FE141E062E081E037D761E070E089
:1001D00080E090E053D622ED41E062E081E02DD74F
:1001E00061E070E080E090E049D661E083E0F0D625
:1001F000FDC11092950010929400F8C1672B21F177
:1002000060E080E0E5D661E070E080E090E036D626
:100210002FE141E062E081E010D761E070E080E032
:1002200090E02CD62CE841E062E081E006D761E066
:1002300070E080E090E022D661E080E0C9D61092C4
:10024000930010929200D2C18091920090919300FD
:10025000892B09F0CBC12DC0672B21F160E080E034
:10026000B7D661E070E080E090E008D62FE141E091
:1002700062E081E0E2D661E070E080E090E0FED5EF
:1002800022ED41E062E081E0D8D661E070E080E0FC
:1002900090E0F4D561E080E09BD6D0939300C093CA
:1002A0009200A4C18091920090919300019709F06F
:1002B0009DC160E080E08CD661E070E080E090E07D
:1002C000DDD52FE141E062E081E0B7D661E070E08A
:1002D00080E090E0D3D520E041E062E081E0ADD65F
:1002E00061E070E080E090E0C9D561E080E07FCF20
:1002F00080918A0090918B00892BA9F0A0918C00AD
:10030000B0918D00CD018F779070892B61F411979A
:10031000B0938D00A0938C008FEF082EF1D6109231
:100320008B0010928A00FE01C431D10508F05EC135
:10033000ED5EFF4F099480918A0090918B00892B8C
:1003400009F44DC080918E0090918F00892B81F42B
:100350008091900090919100019751F4A0918C00B0
:10036000B0918D00A130B10501F180E0082EC8D612
:1003700040918C0050918D004130510581F0012B4E
:1003800071F0DA01B5D6202D81E090E002C0880F2F
:10039000991FCA95E2F7282BDA01022EB1D6809177
:1003A000900090919100019749F480918E00909176
:1003B0008F00019690938F0080938E0080918E0025
:1003C00090918F00079709F011C110928F00109241
:1003D0008E0080918C0090918D000196D2C0C43027
:1003E000D10558F48091960090919700019729F4D7
:1003F0000115110509F0F6C0F9C0B801CE0170DE93
:10040000012B09F4F3C080918C0090918D0001972D
:1004100009F0ECC010928D0010928C00E7C0012B07
:1004200009F4E4C0CA30D10519F482E090E010C0AC
:10043000CB30D10519F481E890E00AC0CD30D10568
:1004400019F481E091E004C02E9731F481E891E045
:1004500090938D0080938C0080918A0090918B0006
:10046000892B09F460C0C2C0D90142D6602D77271C
:100470006170707080E090E050DEA0918C00B091CF
:100480008D0036D6602D669577276170707081E09B
:1004900090E043DEA0918C00B0918D0029D6602DB4
:1004A0006695669577276170707082E090E035DE22
:1004B000A0918C00B0918D001BD6602D669566953D
:1004C000669577276170707083E090E026DEA091DA
:1004D0008C00B0918D000CD6602D62956F707727DF
:1004E0006170707084E090E018DEA0918C00B09193
:1004F0008D00FED5602D62956695669563707727B1
:100500006170707086E090E008DE80918C009091C0
:100510008D00019690938D0080938C0064E170E0D3
:1005200080E090E0ABD420918C0030918D00D90117
:10053000DFD5802D8F3F09F097CF58C0012B09F4EC
:1005400055C080918A0090918B00A0918C00B09151
:100550008D00892B71F0A130B10509F447C08FEFF0
:10056000082ECED510928B0010928A0081E090E088
:1005700008C01197D9F181E090E090938B008093AF
:100580008A0090938D0080938C0030C00C3311054D
:100590002CF461E070E082E090E017C00F3B1105A1
:1005A000E4F061E070E083E090E00FC00C331105EF
:1005B0002CF461E070E080E090E007C00F3B110593
:1005C00064F061E070E081E090E08ADD81E090E03D
:1005D000909397008093960009C010929700109214
:1005E000960004C0B801CE017BDD0DCFDF91CF9125
:1005F0001F910F910895BF92CF92DF92EF92FF92D9
:100600000F931F93CF93DF936C018B01B42EFF24C4
:1006100041E0E42EC0E0D0E06B2D6E218C2DD8D4CB
:10062000EE0C60E0802FD4D484E190E047D484E0E5
:1006300099D4F6949695982F882797958795F80ED4
:1006400061E0802FC5D42196C830D10529F784E117
:1006500090E034D48F2D9927DF91CF911F910F9186
:10066000FF90EF90DF90CF90BF900895EF92FF92B0
:100670000F931F93CF93DF9360E086E0A9D441E00E
:1006800067E070E085E090E0B6DF42E467E070E0AC
:1006900085E090E0B0DF833549F0833751F0813455
:1006A00071F4109267001092660009C081E090E03A
:1006B00002C082E090E0909367008093660040E083
:1006C00067E070E085E090E096DF809166009091B1
:1006D00067001816190654F080916800909169001F
:1006E000892B21F462E0E62EF12C03C056E0E52EC2
:1006F000F12CC0E0D0E000E610E00AC040E067E086
:1007000070E085E090E077DFF80181938F0121961A
:10071000CE15DF059CF361E086E05AD480E090E0DE
:10072000DF91CF911F910F91FF90EF900895CF939C
:10073000DF939CDF61E083E04BD461E080E048D44C
:1007400060916000603F20F08091610086FD07C0ED
:1007500081E090E0909391008093900004C010920B
:100760009100109290007727C1E0D0E06C277D27A0
:100770006170707089E090E0D0DC60916000772754
:10078000769567956C277D27617070708FE090E09B
:10079000C4DC6091600077277695679576956795BC
:1007A0006C277D27617070708CE090E0B6DC609102
:1007B0006000772793E0769567959A95E1F76C2727
:1007C0007D276170707088E090E0A7DC6091600028
:1007D000772784E0769567958A95E1F76C277D27E2
:1007E0006170707080E090E098DC60916000772725
:1007F000B5E076956795BA95E1F76C277D2761702E
:10080000707083E090E089DC609160007727A6E05B
:1008100076956795AA95E1F76C277D2761707070D2
:1008200081E090E07ADC60E070E08091600087FD1C
:1008300002C061E070E082E090E06FDC80916600D1
:100840009091670060916100019709F069C0772776
:100850006C277D27617070708BE090E05EDC6091AA
:1008600061007727769567956C277D27617070709A
:100870008AE090E052DC6091610077277695679579
:10088000769567956C277D276170707086E090E0A3
:1008900044DC60916100772753E0769567955A951F
:1008A000E1F76C277D276170707087E090E035DCA0
:1008B00060916100772744E0769567954A95E1F766
:1008C0006C277D27617070708DE090E026DC609170
:1008D0006100772735E0769567953A95E1F76C27C3
:1008E0007D276170707085E090E017DC6091610099
:1008F000772726E0769567952A95E1F76C277D277F
:100900006170707084E090E008DC60E070E08091DD
:10091000610087FD02C061E070E08EE090E068C099
:1009200077276C277D27617070708BE090E0F5DB96
:10093000609161007727769567956C277D276170B8
:1009400070708EE090E0E9DB60916100772776952A
:100950006795769567956C277D27617070708AE042
:1009600090E0DBDB609161007727B3E076956795D7
:10097000BA95E1F76C277D27617070708DE090E08B
:10098000CCDB609161007727A4E076956795AA9506
:10099000E1F76C277D276170707087E090E0BDDB28
:1009A000609161007727F5E076956795FA95E1F714
:1009B0006C277D276170707085E090E0AEDB609100
:1009C00061007727E6E076956795EA95E1F76C2771
:1009D0007D276170707084E090E09FDB60E070E0E4
:1009E0008091610087FD02C061E070E086E090E0E8
:1009F00094DB80916600909167001816190634F018
:100A00008091680090916900892BC1F0609162002B
:100A1000772780E190E081DB60916300772781E1B7
:100A200090E07BDB60916400772782E190E075DBEA
:100A300060916500772783E190E06FDBDF91CF91D4
:100A4000089560E086E0C4D241E067E070E085E0B0
:100A500090E0D1DD43E467E070E085E090E0CBDD3D
:100A600040E067E070E085E090E0C5DD41E067E0F0
:100A700070E085E090E0BFDD40E067E070E085E099
:100A800090E0B9DD61E086E0A3D264E670E080E04A
:100A900090E0F4D160E086E09BD241E067E070E056
:100AA00085E090E0A8DD44E467E070E085E090E058
:100AB000A2DD40E067E070E085E090E09CDD41E091
:100AC00067E070E085E090E096DD40E067E070E090
:100AD00085E090E090DD40E067E070E085E090E048
:100AE0008ADD40E067E070E085E090E084DD40E092
:100AF00067E070E085E090E07EDD40E067E070E078
:100B000085E090E078DD61E086E062D264E670E046
:100B100080E090E0B3D160E086E05AD241E067E047
:100B200070E085E090E067DD43E467E070E085E039
:100B300090E061DD40E067E070E085E090E05BDD43
:100B400040E067E070E085E090E055DD40E067E080
:100B500070E085E090E04FDD40E067E070E085E028
:100B600090E049DD40E067E070E085E090E043DD43
:100B700040E067E070E085E090E03DDD40E067E068
:100B800070E085E090E037DD61E086E021D20895F5
:100B9000CF93DF93109297001092960010929500D9
:100BA0001092940068E873E180E090E067D160E023
:100BB00084E0BAD161E085E0B7D161E086E0B4D1EC
:100BC00061E087E0B1D160E088E0AED160E089E02B
:100BD000ABD160E08AE0A8D160E08BE0A5D160E015
:100BE0008CE0A2D160E08DE09FD160E083E19CD1F8
:100BF00061E083E099D161E080E096D161E082E03C
:100C000093D161E081E090D161E086E0E1D161E0E3
:100C100087E0DED161E085E0DBD181E090E0909378
:100C2000690080936800C0E0D0E020DD2196C530E7
:100C3000D105D9F7C0E0D0E019DD8091680090912E
:100C40006900892B11F490E005C090E0809160006C
:100C500087FF91E0892F992790936900809368001E
:100C60002196C431D10541F7EAE6F0E02FEF3FEFDE
:100C70002193319340E0EA38F407D1F7892B01F151
:100C800089E090E090938700809386008AE090E06E
:100C900090937500809374008BE090E090937900BE
:100CA000809378008CE090E09093730080937200C2
:100CB0008DE090E09093770080937600C2DE67C06D
:100CC00089E090E090936B0080936A008AE090E066
:100CD00090936D0080936C008BE090E090936F0098
:100CE00080936E008CE090E0909371008093700090
:100CF0008DE090E0909373008093720083E190E028
:100D0000909377008093760060E083E061D161E0AA
:100D100070E080E090E0B2D02FE141E062E081E05D
:100D20008CD161E070E080E090E0A8D02FEF41E04E
:100D300062E081E082D161E070E080E090E09ED0EE
:100D400061E083E045D168EC70E080E090E096D00F
:100D500060E080E03DD161E070E080E090E08ED026
:100D60002FE141E062E081E068D161E070E080E085
:100D700090E084D02FEF41E062E081E05ED161E05D
:100D800070E080E090E07AD061E080E021D11092C4
:100D90008B0010928A0010928F0010928E002FE725
:100DA00030E0D901A5D1802D8F3F21F08FEFD901FF
:100DB000082EA6D12FEF30E0D9019AD1802D8F3F98
:100DC00021F08FEFD901082E9BD12FE731E0D90117
:100DD0008FD1802D8F3F21F08FEFD901082E90D138
:100DE0002FEF31E0D90184D1802D8F3F21F08FEF9B
:100DF000D901082E85D1DF91CF9108956CD0C8DE3E
:100E000096DCFECF1F920F920FB60F9211248F9394
:100E10009F93AF93BF9380919A0090919B00A09174
:100E20009C00B0919D000196A11DB11D80939A0078
:100E300090939B00A0939C00B0939D00BF91AF91B5
:100E40009F918F910F900FBE0F901F9018956091FA
:100E50009A0070919B0080919C0090919D0027E0EA
:100E6000660F771F881F991F2A95D1F72DE730E06D
:100E700040E050E01BD1CA01B9010895AF92BF9282
:100E8000CF92DF92EF92FF920F931F935B016C0161
:100E9000DEDF7B018C01DBDF6E197F09800B910B9C
:100EA0006A157B058C059D05B0F31F910F91FF908E
:100EB000EF90DF90CF90BF90AF900895019751F0E1
:100EC000880F991F880F991F02972FB7F8940197E1
:100ED000F1F72FBF0895789410929A0010929B001A
:100EE00010929C0010929D0083B7826083BF83B7ED
:100EF000816083BF89B7816089BF8EB582608EBDF6
:100F00008EB581608EBD8FB581608FBD85B58460E3
:100F100085BD85B5806485BD3F983E9A329A319AE9
:100F2000309A379A1AB80895282F3327C9018F5855
:100F30009F4FFC019491235A3F4FF90184918823DC
:100F400081F0E82FFF27E25BFF4FE491FF27662344
:100F500029F4808190958923808308958081892B4D
:100F600080830895482F5527CA018B579F4FFC0156
:100F70002491CA018F589F4FFC019491435A5F4FAF
:100F8000FA013491332319F480E090E0089522238C
:100F900081F0233019F48FB58F7704C0243021F409
:100FA0008FB58F7D8FBD05C0253019F485B58F7D38
:100FB00085BDE32FFF27E85AFF4FE491FF2780818B
:100FC00020E030E0892311F021E030E0C9010895EC
:100FD000482F5527CA018B579F4FFC012491CA0106
:100FE0008F589F4FFC019491435A5F4FFA013491FF
:100FF000332311F1222381F0233019F48FB58F7739
:1010000004C0243021F48FB58F7D8FBD05C02530FD
:1010100019F485B58F7D85BDE32FFF27ED5AFF4F6E
:10102000E491FF27662329F48081909589238083AA
:1010300008958081892B80830895CF92DF92EF926B
:10104000FF920F931F93CF93DF93E82EF62EC42EBB
:10105000D22EC0E0D0E007E010E06D2D7727CC2045
:1010600039F40C2E02C0759567950A94E2F706C014
:10107000002E02C0759567950A94E2F761708E2D77
:10108000A7DF61E08F2DA4DF60E08F2DA1DF219627
:1010900001501040C830D10501F7DF91CF911F9169
:1010A0000F91FF90EF90DF90CF900895A1E21A2E5C
:1010B000AA1BBB1BFD010DC0AA1FBB1FEE1FFF1FFC
:1010C000A217B307E407F50720F0A21BB30BE40B4C
:1010D000F50B661F771F881F991F1A9469F7609593
:1010E0007095809590959B01AC01BD01CF0108954D
:1010F000E199FECFBFBBAEBBE09A11960DB2089549
:10110000E199FECFBFBBAEBB0DBA11960FB6F894F6
:0A111000E29AE19A0FBE0895FFCFA6
:00000001FF
